S01B000070705F476E6F6D5F31335F4176746F4E756C2B70756C7365D5
S1130000DEC0189518951895189518951895189593
S1130010189518950150104098018901232BD1F7A8
S1130020089512E813BF06BF00E21EE4F3DF00E008
S113003003BF08950FD1C250B99ABC9A02EE06B913
S113004003E007B900E117E2E5DF02E50FBD00E8D0
S113005008B9C49A00E1E5DF00E2E3DF00E4E1DF90
S113006000E41FE1D7DF00E1DCDFC49800E003BF58
S113007000E61AEECFDF00E61AEECCDF6624772422
S1130080FF2418ECC19888249924AA24BB24DD24D5
S113009012C015B100E024B130E0022B132B212F44
S11300A0220F220B322F800E911EA21EB31E05E1D9
S11300B010E0B0DFD39400E4D01658F38815990506
S11300C0AA05BB052CF48F5F9F4FAF4FBF4F04C0F1
S11300D081509040A040B040FF2021F4C401D501DC
S11300E007E0F02E8C019D01081919092A093B0922
S11300F0013540E0140740E0240740E0340794F160
S113010066247724C49A41E0440E40E0541E488299
S11301105982488059804CE050E060E070E04A0128
S11301205B0148EE53E060E070E073D0801A910AFE
S1130130A20AB30A0881198120E030E080169106F2
S1130140A206B306E4F444245524CC24E0940FEF2F
S1130150E01629F402E803BF01E106BF10C000E085
S113016003BF0DC000E003BFC498C19800E0E02EB7
S1130170102FC3940C2DC02E002309F4FF2401E09A
S1130180600E00E0701E83013801013526E4120779
S113019008F479CF66247724DD2403E0D01608F030
S11301A072CFC49A01E13DDFC198C49800E41CE910
S11301B031DFFF24D394F1CF00008895FECF0FE9FF
S11301C00DBFC0E858D036DFF7DFF6CF0024112486
S11301D01001E0E2EA9592F0001F111F221F331F65
S11301E0001C111C221C331C041615062606370697
S11301F088F3041A150A260A370AECCF001F111FC8
S1130200221F331FA001B101009510952095309550
S11302100895FF27772312F4F16014D0332312F4E6
S1130220F09508D0D3DFF69508F404D0F69508F4D9
S113023009C0089530952095109501951F4F2F4FB3
S11302403F4F089570956095509541955F4F6F4F5E
S11302507F4F0895FA92EA92DA92CA92BA92AA92D7
S11302609A928A927A926A925A924A92BA93AA93E8
S10D02709A938A93089501E008951B
S9030000FC
